:10000000B601092AB80071218413FA30A600A701AD
:10001000EE21A00AA50AA201A30100083805A60046
:10002000640000083805A7002606270538060319CE
:10003000A20A0319A30A2708A600A4030319A5030B
:100040000319A00B10282208042AB616B61EB612F1
:10005000B6192E28B6156920031855280830A300B4
:100060007E20A20DA30B3028B61E6020882084209D
:10007000B61A55205A2022080310042AB616B61EB6
:10008000B61236194828FE39B70036150310042A6F
:10009000361A5028A6003616692003185528260857
:1000A000712003185528B61E042A602088203611B6
:1000B0003612B6113A08840038088417800466287E
:1000C0003A08840038098005841780056728682865
:1000D000042A5A2088200822602084203708B61974
:1000E0000138A2000830A300A20D03185A20031CF7
:1000F000602088208420A30B74285A2088203A0886
:10010000840038080005FF3E3B0884003909632855
:100110003B08840039085D28A400B7172730A300E6
:1001200010309E200330A300E8309E20A3016430ED
:100130009E20A3010A309E202408A928A200250899
:10014000A1002408A000D2212008031DB713B71B6B
:100150000800303EA700071187108710831607118B
:1001600087108710F030860583122708B618D62826
:100170003A30A1009830AD213330A600EB20133087
:10018000A1008830AD21EB206430AC21EB2064303D
:10019000AC212230A600EB202830D5200C30D52011
:1001A0000630D520B6142708D6283614A600361CEB
:1001B000E4288710033C031CE928E9200730A1004C
:1001C000D030AD21031408003614FE3C0319042A74
:1001D0008714A60E361C36100715F0308605260843
:1001E0000F3986040711A60E3618EB283230AC21E1
:1001F00003140800B800841780048413A201201C93
:10020000A20008210319042A08210319042A082935
:100210003808A2060130A000A10100083805220616
:10022000031D0800A00A0319A10F0D290800A5014C
:10023000A400B7172730A30010302A210330A300F1
:10024000E8302A21A30164302A21A3010A302A219F
:1002500024083529A2002508A1002408A000D221E5
:100260002008031DB713B71B0800303EA6003A084C
:1002700084000930A70003104221A60CA70B3C29DB
:10028000031442298413B71D512900083804371D6F
:1002900038068000841700083804031C38068000E4
:1002A0005C2900083804031C38063719380680001A
:1002B0008417380980055C29370D0639A0006521AF
:1002C000A100A00A65210000AD2901308A002008A4
:1002D00082070134993403343934003460340C34E7
:1002E000FD3484178004042AA000A00DA00DA00DE9
:1002F0003830A005813020049F000030A10032304A
:10030000AD211F151F1982291E08A10083161E0882
:10031000042A03178D0083168C130C1483120C0807
:10032000042A03178C0083168C130C1555308D008E
:10033000AA308D008C148C189B290C11042AA3015F
:10034000A200FF30A207031CA307031C042A0330EA
:10035000A100E730AD21A129A101FC3EA000A10927
:10036000031CB829FF300000A0070318B329A00719
:100370006400A10FB2290800A2000130C229A20026
:100380000630C229A80023082102031DC92922081A
:100390002002043003180130031902302805031D20
:1003A000FF30042A1030A600A501A401210DA40DE0
:1003B000A50D2208A4022308031C230FA50203187D
:1003C000E8292208A40723080318230FA507031010
:1003D000A00DA10DA60BD6292008042A1030A800D4
:1003E000A101A001A70CA60C031CFC292208A00750
:1003F00023080318230FA107A10CA00CA50CA40C23
:10040000A80BF2292408042A83130313831264001F
:1004100008008316DF30850085309F00703086002D
:1004200081138701831285018601870107108316D6
:100430000710643083129F218A11DD2A86178316E4
:100440008613FE308312AA200130AA202030AA2071
:100450002030AA204830AA206530AA206C30AA207B
:100460006C30AA206F30AA202030AA202130AA2088
:100470000330A300E830A021FE30AA200130AA20DA
:100480005630AA203130AA205230AA205030AA205B
:100490002030AA207630AA206530AA207230AA2007
:1004A0002E30AA203730AA202F30AA203230AA209E
:1004B0003030AA200130A300F430A021FE30AA2061
:1004C000C030AA20B130AA20B530AA202030AA20FE
:1004D0006B30AA206530AA207930AA202030AA20CB
:1004E0007430AA206F30AA202030AA205330AA20CE
:1004F0007430AA206130AA207230AA207430AA2059
:100500006400061B802A08005830A2000230A300B5
:100510000530840020300220CA002308CB000800E8
:100520000130A000053084000430FA202008C80003
:100530002108C900080000307421BC002108BD005A
:100540000A309F21080001307421BE002108BF003D
:100550000A309F2108000730BA001030B800073079
:10056000BB000830B900A0304020410840204008BE
:1005700040203F0840203E0840204B0840204A08C9
:100580003E200A309F2108000730BA001030B80022
:100590000730BB000830B900A0304020410840209F
:1005A000400840202720BF002720BE002720CB0086
:1005B0002520CA000A309F2108008613831686135F
:1005C00083121E22C8309F216400061FE42AFE30D9
:1005D000AA200130AA20B130AA20B530AA203A3092
:1005E000AA204C30AA206F30AA206730AA202030E1
:1005F000AA20B730AA202030AA203A30AA205030B2
:10060000AA206C30AA206130AA207930AA20FE30BE
:10061000AA20C030AA20B130AA20B630AA203A3091
:10062000AA204C30AA206F30AA206730AA202030A0
:10063000AA205330AA207430AA206F30AA2070302C
:10064000AA20C8309F2164008A11061F3A2B8A1104
:10065000861783168613323083129F2164008A1115
:10066000861E372C8A118613831686133230831226
:100670009F21232BCE0164000A304E028A110318F9
:10068000552B8A1186138316861383120130A3001B
:10069000F430A02186178316861383120130A3003D
:1006A000F430A021CE0A031D3B2BC001C10140083C
:1006B000A0004108A1001F30A3003F30BC218A11D7
:1006C000031DDE2B8A114008A0004108A100043060
:1006D000A200A301D221B2002108B30001303207E9
:1006E000C40033080318013EC500A3228422FE3053
:1006F000AA200130AA204430AA202330AA203D306D
:10070000AA204508A50044088C20FE30AA2002300B
:10071000AA20FE30AA201430AA20FE30AA201430CD
:10072000AA20FE30AA201430AA20FE30AA201430BD
:10073000AA20FE30AA201430AA20FE30AA201430AD
:10074000AA20FE30AA201430AA20FE30AA2014309D
:10075000AA20FE30AA201430AA203F08A5003E0897
:100760008C203030AA206D30AA205630AA20FE30CE
:10077000AA20C030AA205230AA205030AA204D30E2
:10078000AA203D30AA204B08A5004A088C20303012
:10079000AA203030AA207230AA207030AA206D30F2
:1007A000AA20AB2264008A11061EDF2B8A110430B6
:1007B000C007031C572BC10A031D572BE72A8613BA
:1007C0008316861383120130A300F430A021400861
:1007D000CD004008A0004108A100A2010130A30003
:1007E000D221CC00031705308D0003134D08912151
:1007F000031706308D0003134C089121FE30AA2008
:100800000130AA205330AA207430AA206F30AA20C9
:100810007030AA204C30AA206F30AA206730AA205E
:100820006730AA206930AA206E30AA206730AA203B
:10083000FE30AA20C030AA204530AA204E30AA207F
:100840004430AA202030AA205430AA204930AA20BF
:100850004D30AA204530AA203D30AA204508A500E9
:1008600044088C200B30A300B830A021E72A86175B
:1008700083168613FE308312AA200130AA20B130DD
:10088000AA20B530AA203A30AA205030AA206C30D5
:10089000AA206130AA207930AA202030AA20B730BF
:1008A000AA202030AA203A30AA205330AA2074303F
:1008B000AA206530AA207030AA20FE30AA20C030BD
:1008C000AA20B130AA20B630AA203A30AA2045305A
:1008D000AA204E30AA204430AA200330A300E830DA
:1008E000A02164008A11061F7C2C8A1164008A11E1
:1008F000861EA82D8A11712C861383168613053047
:1009000083128921CD0006308921CC004C08A60035
:10091000A701A2010130A300EE21B2002508B30017
:100920004D083207C60033080318013EC700C00156
:10093000C1014008A0004108A1004708A3004608E3
:10094000BC218A11031D642D8A114008A0004108B2
:10095000A1000430A200A301D221B2002108B300FB
:1009600001303207C40033080318013EC500C42219
:10097000FE30AA200130AA204430AA202330AA2029
:100980003D30AA204508A50044088C20FE30AA204E
:100990000230AA20FE30AA201430AA20FE30AA205D
:1009A0001430AA20FE30AA201430AA20FE30AA203B
:1009B0001430AA20FE30AA201430AA20FE30AA202B
:1009C0001430AA20FE30AA201430AA20FE30AA201B
:1009D0001430AA20FE30AA201430AA203F08A50017
:1009E0003E088C203030AA206D30AA205630AA2034
:1009F000FE30AA20C030AA205230AA205030AA20AF
:100A00004D30AA203D30AA204B08A5004A088C2072
:100A10003030AA203030AA207230AA207030AA20AC
:100A20006D30AA200730BA004030B8000230B7005D
:100A30004430362161303621743036216130362120
:100A4000233036213D3036212C3036214508A50093
:100A5000440818212C3036214130362130303621DF
:100A60003D3036212C3036213F08A5003E081821A4
:100A7000303036212C3036216D303621563036213B
:100A80003A3036212C3036214B08A5004A0818216F
:100A900030303621303036212C303621723036213C
:100AA000703036216D3036210D3036210A30362136
:100AB00064008A11061E692D8A110430C007031CC8
:100AC000992CC10A031D992C0730A300D030A02116
:100AD000E72AFE30AA200130AA205330AA20743021
:100AE000AA206F30AA207030AA202030AA205030CF
:100AF000AA206C30AA206130AA207930AA20623066
:100B0000AA206130AA206330AA206B30AA20FE30D0
:100B1000AA20C030AA204530AA204E30AA20443056
:100B2000AA202030AA204430AA206130AA207430A4
:100B3000AA206130AA202330AA203D30AA204508EF
:100B4000A50044088C200B30A300B830A021E72A70
:100B5000861383168613053083128921CD00063053
:100B60008921CC004C08A600A701A2010130A300F6
:100B7000EE21B2002508B3004D083207C600330845
:100B80000318013EC700C001C1016400861EC52DC7
:100B90004008A0004108A1004708A3004608BF2163
:100BA0008A11031DD62D8A11C001C1014008A00081
:100BB0004108A1000430A200A301D221B200210803
:100BC000B30001303207C40033080318013EC500EA
:100BD000C422FE30AA200130AA204430AA202330AB
:100BE000AA203D30AA204508A50044088C20FE30EC
:100BF000AA200230AA20FE30AA201430AA20FE30FB
:100C0000AA201430AA20FE30AA201430AA20FE30D8
:100C1000AA201430AA20FE30AA201430AA20FE30C8
:100C2000AA201430AA20FE30AA201430AA20FE30B8
:100C3000AA201430AA20FE30AA201430AA203F088F
:100C4000A5003E088C203030AA206D30AA205630F6
:100C5000AA20FE30AA20C030AA205230AA2050304C
:100C6000AA204D30AA203D30AA204B08A5004A08F2
:100C70008C203030AA203030AA207230AA20703068
:100C8000AA206D30AA200730BA004030B8000230E8
:100C9000B70044303621613036217430362161305E
:100CA0003621233036213D3036212C30362145087F
:100CB000A500440818212C3036214130362130302F
:100CC00036213D3036212C3036213F08A5003E0824
:100CD0001821303036212C3036216D3036215630F7
:100CE00036213A3036212C3036214B08A5004A08EF
:100CF000182130303621303036212C3036217230F8
:100D00003621703036216D3036210D3036210A30D3
:100D1000362164008A11861A972E8A110430C00287
:100D20000030031C013EC102C8309F21C82D640061
:100D30008A11061EA92E8A1164008A11061BA82E8C
:100D40008A110430C0070318C10AC8309F21C82D7A
:100D5000892EFE30AA200130AA205330AA207430F8
:100D6000AA206F30AA207030AA202030AA2050304C
:100D7000AA206C30AA206130AA207930AA206230E3
:100D8000AA206130AA206330AA206B30AA20073045
:0C0D9000A300D030A021E72A6300CC2E85
:02400E00763DFD
:00000001FF
